:100000000C947401189518951895189518951895CD
:100010001895189518951895189518951895189578
:100020001895189518951895189518951895189568
:100030001895189518951895189518951895189558
:100040001895189518951895189518951895189548
:100050001895189501000000010000000100000043
:10006000010001000100010000000000000000008C
:10007000000001000000010001000000010000007C
:10008000000001000000010001000100010001006A
:100090000000000000000000000001007B2F2A2E5D
:1000A000C2510FEF01BB00E002BB00E00ABB0FE052
:1000B0000BBB0FEF04BB00E005BB31C0EC2FA0E68B
:1000C000B0E00D91102F02E0109FE00DF0E00081F4
:1000D00002BB0FE916E821E0015010402040E1F793
:1000E00000C0000000E002BBE0E6F0E0008111810A
:1000F0000F5F1F4F00831183A0E6B0E0ED91FC91EC
:100100003997E4F207E505BB0FE716E928E9015046
:1001100010402040E1F700C0000000E005BBC89996
:1001200011C06C2F24E530E0062F10E0F90142E108
:1001300050E00E94860100E010E0E0E6F0E000837D
:100140001183DACFC99943C06C2F26E630E0062F21
:1001500010E0F90142E150E00E94860100E010E069
:10016000E0E6F0E0008311831EC0EC2FA0E6B0E0D3
:100170000D91102F02E0109FE00DF0E0008102BB16
:100180000FE916E821E0015010402040E1F700C0DF
:10019000000000E002BBE0E6F0E0008111810F5FAB
:1001A0001F4F00831183A0E6B0E0ED91FC913997D9
:1001B000E4F205E005BB0FE716E928E9015010401D
:1001C0002040E1F700C0000000E005BBA8CFCA99BD
:1001D00043C06C2F28E730E0062F10E0F90142E120
:1001E00050E00E94860100E010E0E0E6F0E00083CD
:1001F00011831EC0EC2FA0E6B0E00D91102F02E09D
:10020000109FE00DF0E0008102BB0FE916E821E04D
:10021000015010402040E1F700C0000000E002BBA8
:10022000E0E6F0E0008111810F5F1F4F0083118332
:10023000A0E6B0E0ED91FC913997E4F20BE405BB48
:100240000FE716E928E9015010402040E1F700C00F
:10025000000000E005BB63CFCB9961CF6C2F2AE88B
:1002600030E0062F10E0F90142E150E00E948601E3
:1002700000E010E0E0E6F0E0008311831EC0EC2F08
:10028000A0E6B0E00D91102F02E0109FE00DF0E02D
:10029000008102BB0FE916E821E001501040204028
:1002A000E1F700C0000000E002BBE0E6F0E0008102
:1002B00011810F5F1F4F00831183A0E6B0E0ED9125
:1002C000FC913997E4F201EC05BB0FE716E928E948
:1002D000015010402040E1F700C0000000E005BBE5
:1002E0001ECF00008895FECF01EA0DBF00E00EBFD3
:1002F000C2E8D0E00E949101002311F00E94A10108
:100300000E944E000E9471010C947101AF93BF9343
:10031000D80105900D9241505040D9F7BF91AF914F
:10032000089501E0089520E006D0E9F708952591A9
:1003300002D0E9F708952D9301501040202F212B72
:10034000089586E793E0FC0105911491FC01329633
:10035000A591B491FC01349625913491422F432B01
:1003600019F0F901E4DF01C0DEDF069613E08C37F7
:0C037000910748F30895020060000000AF
:00000001FF
:00000001FF
